:020000040000FA
:040000008A01422807
:08000800A000030E8301A1001A
:100010000A08A200DF308100AE0B1F28A8012808C3
:1000200087008500FF30AE002908A3002A08A4003D
:100030002B08A5002C08A6002D08A7003A282308A5
:100040002E02031D2428281424082E02031D29280B
:10005000A81425082E02031D2E28281526082E0276
:10006000031D3328A81627082E020319281628086E
:10007000870085000B1122088A00210E8300A00E44
:10008000200E09008F20AC20A2200030AF000730E6
:10009000B00083122F08B1003008B200B208031973
:1000A000B103B2038C1A1408171D522814088C1EB1
:1000B0005728171957281408AF08031D632830085C
:1000C000013A031970288C1E63281408B20803191A
:1000D000B103B203B208031D6328B108031D6328EE
:1000E0008C1E70281408B300B220A9008C1E76283C
:1000F0001408B300B220AA008C1E7C281408B30098
:10010000B220AB008C1E82281408B300B220AC00D1
:100110008C1E88281408B300B220AD004A28831230
:100120008701850199018316071087100711871130
:100130000512851291010F178F160F1605108510E5
:100140000511080083128716960190309700013040
:100150009300920191150800A0308B008316810155
:1001600083120800FF3A0319B72833080800FE304D
:02017000080085
:00000001FF
